:02000000B7281F
:080008001C288207A0342534F6
:10001000A0343534A034703420345034A03430341B
:10002000A034503490345034A0347034A034503460
:100030002034503420345034A500030E8312A40021
:10004000221C2928CA0B2928C90B2928C80B2928B2
:1000500007212A1D2E28B10B33282A11271C3328EB
:10006000B00B33282710A71C3928BF0B3928A7103D
:100070000613271D4128BC0B4128BD0B4128271121
:100080008611A71D4F28B50B4F2810308606FF306C
:10009000061E8030B500B60B4F28A7110612271E8A
:1000A0005528BA0B552827128613A71E6228B40BB1
:1000B0006228203086062D080520B400AD0B62288A
:1000C000A7128612271F6B28B70B6B2827139921BD
:1000D000FF30B1002A15281C7928C20B7928C30BE0
:1000E00079282810AE20221D772876217928A21998
:1000F0008921A21C9728B20B9728A81C84280430B9
:100100000619003086049128AA1C8C280430061990
:100110000230861801309128043006190130061883
:10012000023006118610061086047E30B200A81C2C
:100130009E28C20B9E28C30B9E28A8100000281ED4
:10014000A728C60BA728C70BA728281285150B11AF
:100150008B10240E8300A50E250E09000616803094
:10016000CC00CB0BB128CC0BB128061208008501BE
:1001700007309F0086010313831607308500860130
:10018000640004308100831281019921A0308B002A
:10019000AA012A142A19F528271FD228051CD428B9
:1001A000A721F5280518DA282A18F528A7212A14E6
:1001B0002713F5282A1CF028A7212A10A21CE928B9
:1001C000AC0A03302C02031DF2280230AA06AC014F
:1001D000F228271CED280721F528A030B0002714AD
:1001E0002218CA28FF30B70027172218CA28281853
:1001F000CA28A818CA282819CA282719CA28AA1834
:10020000032905190529851CCA284421CA28CE01BD
:10021000AC01A701A8018601851500308B003030A4
:10022000CD000615061636210612282106112821B2
:100230004E1C1C294E101E29CD0B1129A0308B00FD
:10024000C2010330C300A201A2142810A8140800A0
:10025000A030CB0000002C304D02031831290518C6
:100260004E14CC0B2A29CB0B2A2908002030CB00B6
:1002700000002C304D0203183F2905184E14CC0BFA
:100280003829CB0B38290800AE200611061086103D
:10029000A21C4E29A201221586145129A201A215E1
:1002A0000614CE0100308B003030CD0086100614CD
:1002B0000616362106123621061636210612282188
:1002C000061028214E1C66294E106829CD0B57298F
:1002D000A0308B00FF30C2000230C300A8102814E9
:1002E0008511C6012030C70028160800BC01163051
:1002F000BD00271586150130B4001530AD00A716D6
:100300004030BF00A71406174030BA0027168617E2
:100310000800BC011630BD00271586150630B50053
:100320001930B600A71506124030BA0027168617F6
:1003300008000130A200A701A801AC01023086002C
:100340008515FF30C800C9001A30CA0008002030E7
:06035000B1002A150800AF
:02400E00193F58
:00000001FF
